:030000000219FDE5
:03000B000200AA46
:03002B0002015C73
:03005B000202F6A8
:030073000202E3A3
:1000800002030406080C10182030406080040608A3
:100090000C10182030406080A0C00003070F1F0D17
:1000A0000D04050D050305030302C2AFC0D0C0E077
:1000B000206214E5256009E473E525F4F58AD2622F
:1000C000D0E0D0D0D2AF3285268AC262E526F46075
:1000D0002F30682520720DD0E0D0D0D292D291D2AC
:1000E00090D2AF32D292D291D290206F0C2065097B
:1000F000740AD5E0FDE57B4290D0E0D0D0D2AF329B
:10010000758A00C28DD26201F901B9306805206597
:1001100002C29201B9306805206502C29101B9306E
:100120006805206502C29001B9C29330680A206553
:10013000077408D5E0FDC29201B9C29430680A2064
:1001400065077408D5E0FDC29101B9C29530680A0F
:100150002065077408D5E0FDC29001B9C2AFC2ADF9
:1001600053E6EFC0D0C0E0D2D3D2AFC2CEE52A6012
:100170000720744F152A21C37800790020742EE5DA
:1001800080307E01F430E40278FF53DACF207E0322
:1001900043DA20307E0343DA10C2D8C271E58030E2
:1001A0007E01F430E40279FFC3E89970CB3061033B
:1001B000752A18207403752A18885CD270E86003C9
:1001C000755F0020740DE52B6004152B21D343DAF5
:1001D00001C2D82070024142A85C206102C2702096
:1001E00074367982B70431C3E894F0400374F0F8B0
:1001F000E8C4540F28F87984B703024118C313C325
:10020000138721200802C313200A06C3C898F841A7
:100210001828F8500374FFF88822E52D5406602250
:10022000206B1FE536C333C333F8E564C313C31330
:10023000F9C3952240028922E82522F52250037550
:1002400022FF7882B60459852224A824C3E5249588
:10025000614002A861C3E895634002A8638825E570
:100260006670024193C3E8AA669A5003E8FAE4F97B
:10027000EAC333FBE568F45B29400D2567F8E567C1
:1002800060021567400B41930AC3E5679A50020567
:100290006778FF8826C26FC3E52694F84002D26FC4
:1002A00020CF0AD0E0D0D043E610D2AD32C2CF0585
:1002B0003A7801E52A6005307402152AC3E55C949A
:1002C000014005755F0041D9756000756900E55F03
:1002D0002401F55F5003755FFFD0E0D0D043E610F6
:1002E000D2AD32C2AF53E67F7592FA7593FFC2600A
:1002F000759104D2AF32C2AF53E6EFC2ADC0D0C0E9
:10030000E0C0F0D2D3D2AFA8FBA9FCC2D8307102B2
:10031000615D53DACF207E0343DA10307E0343DA87
:1003200020D271E580307E01F420E4026134882718
:100330008928A18A53DACF207E0343DA20307E0356
:1003400043DA10C2D8C271307402A1767800E58019
:10035000307E01F430E402A176885CA15E53DACFEE
:10036000207E0343DA20307E0343DA10C27120611D
:1003700002813653DACF207E0343DA10307E034306
:10038000DA20C2D8D27188578958C3E89555F8E960
:100390009556F97B007E087A00C3E8948CE99400B6
:1003A0005005755B008128882178A2E6A821605558
:1003B000C3E894C8E994005008E4D2E4FB7A0A81C7
:1003C00003C3E89468E994015008E4D2E3FB7A0F90
:1003D0008103C3E894D0E994025008E4D2E2FB7AA6
:1003E0001E8103C3E894A0E994055008E4D2E1FB20
:1003F0007A3C8103C3E89498E994085008E4D2E079
:10040000FB7A787E00C3E89559FCE9955AFD30E700
:100410000AECF42401FCEDF43400FD755B00C3EC40
:100420009AED9E5003755B018859895A8557558509
:1004300058567802A15EC3E89527F8E99528F93067
:100440007C02A142307B02A142307A02A13B20759E
:10045000028159E9FDE8FC8178E9C313F9E813F852
:10046000307902A13BE9C313F9E813F8307802A10F
:0F0470003BE9C313FDE813FC20612CC3EC941C83
:10047F00ED94024002818FED701EC3EC94C85018AA
:10048F000529E52970021529C3E529940A5002A10F
:10049F0076755C00D270A176E529600215297888FF
:1004AF00E6F97400207F087896B90302789EE62457
:1004BF00FAFEE43400FFC3EC9EFCED9FFD9208B9F9
:1004CF000310A2085007207609D27681E130760218
:1004DF00C276A2085016B9030DECF42401FCEDF41A
:1004EF003400FD0204FB78007900A142B90315EC3A
:1004FF0033FCED33FDC3EC940AFCED9400FD500486
:10050F007C007D00C3EC94FFED9400400678FF79EA
:10051F0000A142EC8572F0A4C5F0A2F733F8790080
:10052F00400302055E78FF790002055EE9C313F907
:10053F00E813F8307C0EE9600278FFC3E81338F84F
:10054F00E43400F9C3E894FFE99400400278FF888F
:10055F005CD270206102A176741FF4552F4BF52FDA
:10056F00C274EB7002D274752A18307403752A0A9C
:10057F00306102A18A20740353DAFE207403752BB5
:10058F0006D0F0D0E0D0D0D2AD43E61032790102E0
:10059F0005BA79030205BA790A0205BA791E02056E
:1005AF00BA79640205BA79C80205BA7817E4D5E0BA
:1005BF00FDD8FAD9F6227A147B780205E17A107BFE
:1005CF008C0205E17A0D7BB40205E17A0B7BC80240
:1005DF0005E1E573D5E001227902E4C294D5E0FD8F
:1005EF00C291D5E0FDD291D5E0FDD294D5E0FDE9E1
:1005FF0020E002C29230E002C290E573D5E0FDE93F
:10060F0020E002D29230E002D2907496D5E0FDD96C
:10061F00C9EAF8D5E0FDD8FBDBB8C29422C37C0051
:10062F007D0075F00005F0EA33FAEB33FB50F6EB83
:10063F0013FBEA13FAC3E9FFE8FEE89AF8E99BF91E
:10064F005004EFF9EEF8B3EC33FCED33FDD5F0DFEA
:10065F00EDF9ECF822E889F08A20D2D4F8A9F07BE2
:10066F000030F70B7BFFF42401F8E9F43400F9E8CC
:10067F008520F0A4ADF0F8E98520F0A4AFF0FEEDF1
:10068F002EF974003FFA7C04C3EA13FAE913F9E870
:10069F0013F8DCF48BF030F70AE8F42401F8E9F4EE
:1006AF003400F9E889F0C2D4F8A9F0227882B604B0
:1006BF0003020716C3E55C940140030206E085229E
:1006CF0024E4F544F545F546F547F548C26E0207B3
:1006DF00167882E6FCD26EE522F523783879C7AA20
:1006EF0040AB41C3EB13FBEA13FAEC146013C3EBFB
:1006FF0013FBEA13FAEC14146007C3EB13FBEA13B2
:10070F00FAD12C8844894522C3E5449523F8E54561
:10071F009400F9500CC3E89480E994FF4016020747
:10072F0047C3E8947FE994005003020747787F7925
:10073F0000020747788079FF8849894A22E54925D1
:10074F0046F8E54A3547F9854A20E4300701F43584
:10075F0048FA30E709C3EA94F04015020785C3EA67
:10076F00940F500302078578FF79FF7A0F020785F0
:10077F00780079007AF0C3E5249561500AC37401BB
:10078F009524500B0207A3E54A20E70E0207A3E5C5
:10079F004A30E706884689478A482278A5E6FAC391
:1007AF00E54933F8E54A33F9D164E930E70BC3E89B
:1007BF009480E994FF4013E1DDC3E8947FE994004E
:1007CF005002E1DD787F7900E1DD788079FFE82064
:1007DF00E715C3E52398F84009C3E89401400302E5
:1007EF0008047801020804E8F424012523F84003E3
:1007FF0002080478FF884B2278A6E6FAA847A94892
:10080F00120664E930E70CC3E89401E994FF40163F
:10081F00020839C3E894FFE99400500302083978BD
:10082F00FF7900020839780179FFE920E715C3E560
:10083F004B98F84009C3E89401400302086078011F
:10084F00020860E8F42401254BF8400302086078A1
:10085F00FF88242278FF20692879A1E76023E541EA
:0E086F00601F74FF8541F0848539F0306A0304
:10087D0075F005A4F8C5F0600278FFC3E8956450E3
:10088D0002A864886322C3E5409440E5419401E5E4
:10089D006350031401A4046002F563220208AC2224
:1008AD0075E890227883E6FF30EDF9A8BDA9BE0565
:1008BD0070C3E57094084052757000E9FA79A0E7AD
:1008CD006044EA7007E571601B0208E5C3E89571A5
:1008DD006010E5715006600C140208F10460F90215
:1008ED0008F1E571F571C39458401B7561C0C3944F
:1008FD00044013756180C39404400B756140C3942B
:10090D0004400375610075BB0322E561241050029C
:10091D0074FFF5617982B70402213EC3A861E52415
:10092D00985002A824C3E895634002A863882588DF
:10093D0026E570B4070375BB1022743279A787F0D2
:10094D00A4C5F0A2F733F8C3E895614002A8618809
:10095D00228824882588268864227540007541F0F8
:10096D0022C2AF75C820A8CCA9CDAA3A30CF010AB2
:10097D0075C824D2AFAB3BAC3C883B893CC3E89BEC
:10098D00F8E99C206908F9306602417F21D9AD3D17
:10099D008A3DF9EA9DFA600678FF79FF21BEAE3EE9
:1009AD00AF3F8B3E8C3FA83BA93CC3E89EF8E99F27
:1009BD00F9C3E54113FBE54013FAE82AF540E93B9D
:1009CD00F54150067540FF7541FF4126AA40AB41E8
:1009DD00AC40AD417E047F02C3EB9404400D1E1F5D
:1009ED00C3EB94084005206A021E1FC3ED13FDECF6
:1009FD0013FCDEF7C3EA9CFAEB9DFBEF6009C3E93C
:100A0D0013F9E813F8DFF7EA28FAEB39FB8A408B84
:100A1D004150067BFF8B408B41C3EB94025002D2B9
:100A2D00663069047F0341517892E6FFC3E5379440
:100A3D008240110FC3E53794A040010FC3EF940618
:100A4D0040027F057E02E541C4540FF9E541C454CF
:100A5D00F0F8E540C4540F28F8C3E89EFAE9940075
:100A6D00FB4009C3EA9402EB940050047A02E4FBC4
:100A7D0041CBAA40AB41EBC4FEEAC4540F4EFCC3BC
:100A8D00EA9CFAEB9400FBC3E813C313F8EA28FAC7
:100A9D00EB3400FB8A408B41C3EB94024002C266EB
:100AAD007802EBC4FE7B00EAC4540F4EFAC3EA98F9
:100ABD00FA4005C3940250027A027892E6FF306044
:100ACD000241CB855192855293D26043E680C3E4B7
:100ADD009AF8E49BF93066026157E8FAE9FBD3E92D
:100AED0013FDE813FC88518952C3EF94036038EF6E
:100AFD0020E00DE82CF8E93DF9ECFAEDFB020B20B6
:100B0D00E828F8E939F9C3E82402F8E93400F97A5C
:100B1D00FE7BFFC3EF9403400E8A538B54884D899F
:100B2D004E8C4F8D50618B885389548A4D8B4E8CD2
:100B3D004F8D503069127553F07554FF754FF07528
:100B4D0050FF7551F07552FF618BE8FAD3E813FC35
:100B5D008851C3EF94036020EF20E007E82CF8ECF8
:100B6D00FA6177E8282402F87AFEC3EF940340086F
:100B7D008A53884D8C4F618B88538A4D8C4FE56815
:100B8D00C3335002646BF5683060026195753402B1
:100B9D00D26043E680E52D54066034A840A941C3D8
:100BAD00E913F9E813F8C3E913F9E813F830690408
:100BBD00E92440F9C2AF53E67F759100C3E498F57F
:100BCD0094E499F595759104D26043E680D2AF22F5
:100BDD00D264754300752000306C03752040020B04
:100BED00FCD264754300752040306C03752000788D
:100BFD00017901206620E52D54066002C264791446
:100C0D00E541C313700104F8C39414400278143005
:100C1D006904781B791B206010E543600C30690373
:100C2D00D53404D26D81A7719D0543E59BF45440E5
:100C3D00B52002819130690908C3E89940011881F6
:100C4D002320640A08C3E899400261FC8123C26431
:100C5D00C2AF53E67F75910030661275940075959D
:0F0C6D00F8759104D26043E680D2AF61FCE54197
:100C7C007EFFC3334005C3334001FEC3E49E75942D
:100C8C0000F595816EC3E5339401500261FC30642C
:100C9C000261FCD80281A58123C26DC2AF53E67FED
:100CAC00759100855394855495759104854D928565
:100CBC004E93D26043E680D2AFE52D5406600820F7
:100CCC006A020533020CE3306D0D206C0A206407B8
:100CDC00158115810215AD2278003064027801E58A
:100CEC003775F007A4F9E5F028F5F0E9A2F013A2A6
:100CFC00F113A2F213F537C394785003753778C308
:100D0C00E53795384008D265D292D291D2903060B6
:100D1C0002A11A854F92855093D26043E68022D26D
:100D2C00A0207D16C2AF754202C294D293306202EB
:100D3C00C290D2AF759F10020F27C2AF754202C28C
:100D4C0094D295306202C292D2AF759F10020F27D7
:100D5C00C2A0307243207D20C2AF75420390013A8D
:100D6C00757B10D290C295306204C291A17CD29452
:100D7C00D2AF759F20020F27C2AF75420390013A84
:100D8C00757B10D292C293306204C291A19CD29412
:100D9C00D2AF759F00020F27207D17C2AF7542039B
:100DAC00900115D290306202C291D2AF759F200291
:100DBC000F27C2AF754203900115D292306202C266
:100DCC0091D2AF759F00020F27D2A0207D16C2AF23
:100DDC00754204C293D295306202C291D2AF759F14
:100DEC0000020F27C2AF754204C295D29330620243
:100DFC00C291D2AF759F20020F27C2A03072432040
:100E0C007D20C2AF754205900129757B08D291C235
:100E1C0094306204C292C126D293D2AF759F100255
:100E2C000F27C2AF75420590014B757B20D291C242
:100E3C0094306204C290C146D295D2AF759F100215
:100E4C000F27207D17C2AF75420590010BD2913050
:100E5C006202C292D2AF759F10020F27C2AF7542C9
:100E6C000590011FD2913062EBC290D2AF759F10EA
:100E7C00020F27D2A0207D16C2AF754206C295D2B2
:100E8C0094306202C292D2AF759F20020F27C2AF7C
:100E9C00754206C293D294306202C290D2AF759F53
:100EAC0000020F27C2A0307244207D20C2AF7542D1
:100EBC000190014B757B20D292C293306204C29098
:100ECC00C1D0D295D2AF759F00020F27C2AF754229
:100EDC0001900129757B08D290C295306205C292AF
:100EEC00020EF1D293D2AF759F20020F27207D17EF
:100EFC00C2AF75420190011FD292306202C290D2F1
:100F0C00AF759F00020F27C2AF75420190010BD243
:100F1C0090306202C292D2AF759F20C265229001BE
:100F2C0009757B00D292D291D290C293C294C29591
:100F3C00C26222788076090876090876040876FF62
:100F4C000876030876FF08760A0876030876010807
:100F5C007601788C76010876FF0876FF0876FF0814
:100F6C0076FF0876FF0876030876FF0876FF08768A
:100F7C00FF0876250876D00876280876500876047F
:100F8C000876FF08760208760008767A0876FF085D
:100F9C007601087601087600087603087600227838
:100FAC0087E6FFC272BF0302D2727888E6C394034D
:100FBC006008C27DE630E102D27DC27E7889E630DF
:100FCC00E102D27EC3EF94026008758E01D27302E7
:100FDC000FE3758E00C273227880E6149000809324
:100FEC0078A5F67881E6149000809378A6F678863A
:100FFC00E61490008D9378A7F67886E6F539C394BD
:10100C00025003753902789CE67538FFB4020375FB
:10101C0038A0B4030375388278A3E61490009A9331
:10102C00F566120F2A22227896E6FA7897E6FB7874
:10103C0088E6B40305C3EB940EFB307F047A007B87
:10104C00FFC3EB9AFCC3948250027C82757200053C
:10105C0072EC8572F0A4C3E5F0947D40F222D27F4D
:0E106C0011331205AB1205AB7A007B007C102D
:10107A001205A1E55C2AFA74003BFBDCF37C04C38D
:10108A00EB13FBEA13FADCF7FEC27F113322757CFD
:10109A0000757D00E5EF20E6037520000520903FEE
:1010AA00FFE520146006901DFF146000930460039E
:1010BA0075EF1653D9BF7581C043FF8012059C7521
:1010CA00EF0643B203E5B3240220E70DF521E5E379
:1010DA0020E0068521B343E301120F2A7580FF75CC
:1010EA00A40075F1D475D4EF75908775A54075F293
:1010FA00FF75D5BF75A60175E24275DB4675EA0232
:10110A00120F2AE4F8F6D8FD756801120F3F12157E
:10111A00FE78988673753001C2AF1205B51205C5FF
:10112A001205AB1205CC1205AB1205D31205ABC2E0
:10113A00AF757C00757D0078FA79FA308407D9FB9F
:10114A00D8F7021C00120FAB120FE41132113378D8
:10115A00988673120F2A75881075890275C82475C6
:10116A00910475D84075A82275B80275E690759BEA
:10117A0080759D0075D10E75BC5875BB0375BA1183
:10118A0075E88012059CD2AF1208A975360053DAA9
:10119A00CF207E0343DA20307E0343DA1043DA019C
:1011AA00C2D8C2711205B5D2617B037A0CE55B70B5
:1011BA00077A0CDB030211391205AB207003021106
:1011CA0039C270E55CC3940240E1E52F541F855E85
:1011DA005DF55EB55DD5DAD5C26153DACF207E03FF
:1011EA0043DA20307E0343DA10C2D8C27178A2E60D
:1011FA007008D274E52F54E0F52FC27575290012D4
:10120A0005B0307409C3E529940A4002D275120563
:10121A00A178023074027800C3E55C9840F0C2AF4E
:10122A001205C51205C51205C5D2AF1205B5754C12
:10123A00007888E6B40302612E1205A1788CE6C311
:10124A009401500302132EE530C394015003021394
:10125A002E757CA5757DF1207435C3E55C94FF502D
:10126A000302132EC2AF1205DAD2AF1205B0C3E5DC
:10127A005C940150EFC2AF1205C51205A61205C54E
:10128A00D2AF1205B0C3E55C94FF40E90217B67FFE
:10129A0002D27F11331205B0C2AFC27F1133AE5CE6
:1012AA00C3E55C947FD2AF5002613E12059CC2AF87
:1012BA001205DAD2AFDFDA116AC3EE7897F61205B1
:1012CA00B51217397F0AD27F11331205B0C2AFC2E5
:1012DA007F1133AE5CC3E55C947FD2AF50E6120552
:1012EA009CC2AF1205C51205A61205C5D2AFDFD63C
:1012FA00116AEE24037896F6F87997E7C394824048
:10130A0003985006E824827897F61205B512164C0F
:10131A001217681205B01133C3E55C94FF500241FD
:10132A005B0217B6757C00757D00C3E55C954C4081
:10133A0003855C4C1205B078017988E7B40302781A
:10134A0005C3E55C984002413BC2AF1205DA1205BB
:10135A00DA1205DAD2AF1205B5753000E4F531F5C7
:10136A00320531E531F4703F0532789AE67819147E
:10137A006012783214600D787D14600878FA14606F
:10138A0003753200C3E53298401D120F2A12059CDC
:10139A00153275310078998673C2AF1205DAD2AF69
:1013AA00789886731205B01205A6E52A700530747E
:1013BA0002213978012074027806C3E55C9840A1BD
:1013CA007888E6C3940360031205B0E52A70030225
:1013DA001139C2AF120F2AE4F522F523F524F525B7
:1013EA00F526F567D2AF7885E6C333F565E4F544AB
:1013FA00F545F546F547F548F570F52CF52DF53721
:10140A0075700875BB1012059C1208AD30EDFDA869
:10141A00BDA9BEE97001F888711208B17570087526
:10142A00BB10120FABC2AF7561FF1209478522616B
:10143A00852262852263D2AF752201752401752542
:10144A0001752601856069756A017888E6B4030723
:10145A00C27D307602D27DD268D269753300120E0F
:0D146A007F120EB012096712096E12096799
:1014770012096E120967120BEE1206BB120CE41268
:101487000D2B12096E120BDD306E03120717206643
:1014970003120863306603120893120CE4120D5C02
:1014A70012096E120BEE306E0312074C120CE41287
:1014B7000DD512096E120BDD306E031207AA120C3E
:1014C700E4120E0612096E120BEE306E03120807B5
:1014D700120CE4120E7F12096E1208AD120BDD1208
:1014E7000CE4120EB01208B112096E30693285642D
:1014F70061856462856069756A0179187A0CC3E54C
:101507003399400FC269D26A8A35856461856463FD
:10151700021527C3E55C9401400302147D0215B54B
:10152700306A25206C22E535147006C26AD26B81B9
:101537007DF535C3E55C9401400302147D7888E6A8
:10154700C3940360030215B575360078FA79A4E7EA
:1015570060027803C3E55F985054307404E52A604D
:101567004D7888E6B40317207D05207607A18530DE
:101577007602A185206C07D26C85646181BC78F006
:10158700306C058564617820C3E541985002817D00
:10159700306C1BC26CC27D307602D27DD26A753543
:1015A70012856461817D0536E55C6002A1B87536F8
:1015B70000C2AF120F2A7887E6FE7602120FAB78C9
:1015C70087EEF6E4F522F523F524F525F526F565EE
:1015D700752C00752D00D2AF1205B0120F2A78A412
:1015E700E66006C292C291C290307409C3E5369490
:1015F70004400221396166901A0D782012168EE593
:1016070020B4550CA312168EE520B4AA0302162C9B
:10161700757CA5757DF1120F3F12164C757C007510
:101627007D0002164B901A0378807B0A12168EA350
:1016370008DBF9901A0F788C7B1912168EA308DB3A
:10164700F9901A2822C2AF1216D11216AE901A00BC
:10165700740E121693A37409121693A37415121617
:1016670093901A0378807B0A121692A308DBF990ED
:101677001A0F788C7B19121692A308DBF91216E45D
:101687001216C2901A2822E493F622E6438F0153DA
:101697008FFDFFC3E583941C400122EF857CB7854E
:1016A7007DB7F0538FFE22438F02438F01857CB7AE
:1016B700857DB7901A0DF0538FFC22901A0D745543
:1016C700D193901A0E74AAD193227A3079D07820C8
:1016D700901A40D18EE520F709A3DAF7227A3079FC
:1016E700D0901A40E7D19309A3DAF922AB74A87511
:1016F700BB01027980BB02027981BB03027982BBFD
:1017070004027984BB05027986BB06027992BB077E
:10171700027987BB080279A3BB0902799CBB0A023D
:101727007988BB0B027989E8F7227C051205B5DCBD
:10173700FB22C2AF1205C51205CC1205D31205DA7A
:101747001205A61205C51205CC1205D31205DA1229
:1017570005A61205C51205CC1205D31205DAD2AFBC
:1017670022C2AF1205DA1205D31205CC1205C51233
:1017770005A61205DA1205D31205CC1205C5120506
:10178700A61205DA1205D31205CC1205C5D2AF226F
:10179700AE74AF75C2AF1205C51205C51205C512E5
:1017A70005A6DEF21205DA1205A6DFF8D2AF22F19E
:1017B70039F131F131757401757501757600F1975D
:1017C7007C05AD5C1205B5C3ED955C70F5C3E55CB2
:1017D7009401400AC3E55C94FF40330217F2D1F34A
:1017E700D14CF139C2AF75EF16F131DCD50576C3AF
:1017F700E5769403500280C61217310575E5741417
:1018070090009F93F808C3E57598500280AD1217B2
:10181700311217310574C3E574940C500280991284
:0D1827000F3F12164CC2AF75EF16121731AD
:0319FD000210983D
:101A00000E0915090904FF03FF0A03010155AA0184
:101A1000FFFFFFFFFF03FFFFFF25D0285004FF0259
:091A2000007AFF0101000300FF40
:101A400023484B696E67323041232020202020201C
:101A500023424C48454C4923463333302320202031
:101A60002020202020202020202020202020202076
:101C0000C2AFC2D353D9BF7581C043B20343FF8073
:101C1000752438752503B1DC7529A5752AF175E29F
:101C20004043F11053A4EF75D4FFD2847DFA7803BA
:101C300079E67C10752200752300901DE97B0675FE
:101C400024987525013084028145208408D8FBD969
:101C5000F9DCF781B7308408D8FBD9F9DCF781B714
:101C6000B19CE493A3C39A6004DDC381B7DBDBB10D
:101C70008E6002812E7B08E493FAA3B16FDBF87AC1
:101C800030B16F752200752300B18EEAFCEBFDC305
:101C9000ED94FE400EB18E8A278B28ED30E0048A49
:101CA000828B83B18E7AC270D8C3ED94FE601950D6
:101CB000CEBD002BEC600F7520007521FF7529004B
:101CC000752A000200008100A827A9280809D80465
:101CD000D90281DCB192EA89AAF281CE0D81A3C337
:101CE000ED94035053EDA2E092007AC5C3E58294CF
:101CF00000E583941C508A200010438F02438F011B
:101D00008529B7852AB7F0300029A827A92808090E
:101D1000438F01538FFDD804D902A133C3E58394C7
:101D20001C4003A3A11689AAE28529B7852AB7F02A
:101D3000A3A116538FFC817F7AC1BD030CE493A34A
:101D4000FAB153DCF8B14B817F8181AA22AB23B178
:101D50006FEBFAEA6222752608C3E52313F523E543
:101D60002213F52250066323A0632201D526EAB18F
:101D7000DCB1DC75260AEAF4200102D284300102CB
:101D8000C284B1DCC3134002C201D526EB22B1925A
:101D9000EAFB208402A192308402A197752608AE46
:101DA00024AF25C3EF13FFEE13FEB1E0B1DCC3EAAD
:101DB000133084024480FA30E703632201C3E52331
:101DC00013F523E52213F52250066323A0632201B5
:101DD000D526D9E52265236523F52222AE24AF2539
:101DE0000E0FDEFEDFFCD20122424C48656C6934E6
:071DF000373164F3300601F6
:00000001FF
